:020000040000FA
:10000000B2EF00F0F76A140FF66E000EF722090047
:10001000F5501200536F6E6172204D555820762EA8
:10002000310A0D00F76A340FF66E000EF722090050
:10003000F5501200417574686F723A20416E647217
:1000400065772057696C736F6E20352F32303036EC
:100050000A0D0000F76A640FF66E000EF722090021
:10006000F55012007265636F6E6E73776F726C6419
:100070002E636F6D0A0D0000F76A880FF66E000E92
:10008000F7220900F5501200736F6E6172313A2049
:1000900025730A0D0000F76AA60FF66E000EF72210
:1000A0000900F5501200736F6E6172323A202573A9
:1000B0000A0D0000EA6A120EE96EEF500DE0020E22
:1000C000016E006A002EFED7012EFBD7970E006E40
:1000D000002EFED7EF2EF3D7F2EF00F0080E006EE1
:1000E000928680A6FED7116A008E0ED0009E0CD09C
:1000F000D89080A6D8801132008C06D0009C002EAB
:10010000F7D711C001F00BD03F0E00BE110E016EEB
:10011000012EFED700BEEAD700BCF0D7E9D7000C0D
:10012000080E006E928280A2FED7116A008E0ED059
:10013000009E0CD0D89080A2D8801132008C06D0BE
:10014000009C002EF7D711C001F00BD03F0E00BE6F
:10015000110E016E012EFED700BEEAD700BCF0D70B
:10016000E9D7000CF86AD09EEA6AE96AC29CC29E8E
:10017000C150800B7F09C16E700ED36EB8960C0E05
:10018000AF6E220EAC6E900EAB6E929089909290F4
:100190008990116A115036DF112A006E00509EA816
:1001A000FED7AD6E0F0E115CF5E1116A11503ADF0A
:1001B000112A006E00509EA8FED7AD6E1E0E115C77
:1001C000F5E1116A115046DF112A006E00509EA819
:1001D000FED7AD6E120E115CF5E1040E116EFA0E33
:1001E000126E68D7112EFBD79294898477DF01C0F5
:1001F00006F00650520804E071DF01C006F0F9D79E
:100200006DDF01C007F06ADF01C008F067DF01C0E1
:1002100009F00A6A116A11502FDF112A006E00508E
:100220009EA8FED7AD6E080E115CF5E1EA6A070ED6
:10023000E96E000EEF1008E09EA8FED7EFCFADFFED
:10024000E92AD8B4EA2AF5D70A0E9EA8FED7AD6EE1
:100250000D0E9EA8FED7AD6E9294899492908980DF
:100260005FDF01C006F00650520804E037DF01C02E
:1002700006F0F9D755DF01C007F052DF01C008F0E2
:100280004FDF01C009F00A6A116A115004DF112A18
:10029000006E00509EA8FED7AD6E080E115CF5E111
:1002A000EA6A070EE96E000EEF1008E09EA8FED77E
:1002B000EFCFADFFE92AD8B4EA2AF5D70A0E9EA8F7
:1002C000FED7AD6E0D0E9EA8FED7AD6E92908990B2
:0402D0008BD70300C5
:020000040030CA
:0E00000000C90F1E0080850003C003E003400E
:00000001FF
